:020000040800F2
:10000000001000206D100008B9100008B910000899
:1000100000000000000000000000000000000000E0
:10002000000000000000000000000000B9100008FF
:100030000000000000000000B9100008B91000081E
:10004000B9100008B9100008B9100008B91000086C
:10005000B9100008B9100008B9100008850D000893
:10006000B9100008B9100008B9100008B91000084C
:10007000B9100008B9100008B9100008B91000083C
:10008000B9100008B910000800000000B9100008FD
:10009000B9100008B9100008B9100008B91000081C
:1000A000B9100008B9100008B9100008B91000080C
:1000B000B910000800000000B9100008000000009E
:1000C0005FF808F180B588B000AF78600023FB616D
:1000D0000023BB6100237B6100233B610023FB60A5
:1000E000654B5B680C221340FB61FB69042B07D056
:1000F000082B09D0002B31D17B68604A1A6031E0AF
:100100007B685E4A1A602DE05B4B5A68F0239B03C4
:100110001340BB61584B5A6880235B0213407B61DC
:10012000BB699B0C0233BB617B69002B05D1BB69AA
:10013000534A5A437B681A6014E04F4BDB6A0F2224
:10014000134001333B614D48396901F0F3FB031C57
:100150001A1CBB695A437B681A6003E07B68474AF4
:100160001A60C046444B5B68F0221340FB61FB6998
:100170001B09FB61434AFB69D3181B78DBB2FB60A8
:100180007B681A68FB68DA407B685A603A4B5A68A9
:10019000E023DB001340FB61FB691B0AFB61394A6A
:1001A000FB69D3181B78DBB2FB607B685A68FB687D
:1001B000DA407B689A60304B1A6B80235B001340F7
:1001C00003D17B68304ADA6010E02B4B5A688023F9
:1001D000DB01134005D17B689B685A087B68DA60B5
:1001E00004E07B689B689A087B68DA60224B1B6B93
:1001F0004022134003D17B68244A1A6103E07B68E4
:10020000802212021A611C4B1B6B1022134003D177
:100210007B681A4A5A6103E07B681A687B685A61F6
:10022000154B1B6B0322134004D17B689A687B68D3
:100230009A611EE0104B1B6B03221340012B04D16B
:100240007B681A687B689A6113E00B4B1B6B032277
:100250001340022B04D17B68802212029A6108E0CD
:10026000054B1B6B03221340032B02D17B68034A0F
:100270009A61BD4608B080BD0010024000127A00AD
:1002800000093D0000000020809FD5001280000082
:1002900080B582B000AF78600A1CFB1C1A70FB1C92
:1002A0001B78002B06D0084B074A51697A680A432D
:1002B0005A6106E0044B044A52697968C9430A400E
:1002C0005A61BD4602B080BD0010024080B582B0C8
:1002D00000AF78600A1CFB1C1A70FB1C1B78002BFB
:1002E00006D0084B074A91697A680A439A6106E08A
:1002F000044B044A92697968C9430A409A61BD4631
:1003000002B080BD0010024080B582B000AF7860BE
:100310000A1CFB1C1A70FB1C1B78002B06D0084B18
:10032000074AD1697A680A43DA6106E0044B044A55
:10033000D2697968C9430A40DA61BD4602B080BD1E
:100340000010024080B582B000AF00F0BFFFC023B4
:10035000DB02181C0121FFF79BFF3B1CFF221A60E8
:100360003B1C00221A713B1C0022DA713B1C032249
:100370005A719023DA053B1C101C191C01F05CF823
:100380003B1C01221A603B1C01221A713B1C0022FB
:100390009A713B1C0022DA71164A3B1C101C191C76
:1003A00001F04AF83B1C02221A603B1C01221A7120
:1003B0003B1C00229A713B1C0022DA710D4A3B1C47
:1003C000101C191C01F038F83B1C38221A603B1C29
:1003D00001221A713B1C00229A713B1C0022DA7127
:1003E000044A3B1C101C191C01F026F8BD4602B043
:1003F00080BDC0460004004880B586B000AF082329
:10040000FB18992212021A600823FB1800221A71A5
:100410000823FB180022DA719023DA050823FB1861
:10042000101C191C01F008F801200121FFF74EFFF4
:1004300000200F2101F0E2F91023FB18992212028B
:100440001A601023FB1800221A711023FB180822CF
:100450005A711023FB1801229A711023FB18181CE3
:1004600001F030F93B1D07221A703B1D00225A7023
:100470003B1D01229A703B1D181C01F007FABD4676
:1004800006B080BD80B58AB000AF78600823FB1845
:10049000181CFFF717FE0823FB185B68181C094996
:1004A00001F048FA031C1A1C7B6853437B6202E08C
:1004B0007B6A013B7B627B6A002BF9D1BD460AB0A7
:1004C00080BDC0461027000080B58AB000AF8023F1
:1004D0009B03181C0121FFF717FF80239B02181CA8
:1004E0000121FFF7D5FE9023DB05181C092104220A
:1004F00001F098F89023DB05181C0A21042201F072
:1005000091F82023FB18181C01F028F82023FB1871
:10051000C022D2001A602023FB1802221A71202365
:10052000FB1801229A719023DA052023FB18101C76
:10053000191C00F081FF3B1D80225203DA603B1D35
:1005400000225A603B1D00229A603B1D00221A6166
:100550003B1D00225A613B1D00229A613B1D084A47
:100560001A60084A3B1D101C191C00F0A7FD054B22
:10057000181C012100F008FEBD460AB080BDC0462F
:100580001F1262C00054004090B585B002AF021C3B
:10059000FB1D1A70FB1D1B789AB20B4980235C046B
:1005A00080239B010093081C111C0122231C00F0D6
:1005B00025FEC046044B181C022100F061FE031EFC
:1005C000F8D0BD4603B090BD0054004090B585B052
:1005D00002AF021CFB1D1A700E4A80235C048023AC
:1005E0009B010093101CC0210122231C00F006FE79
:1005F000084AFB1D1B78101C191C00F033FEC04676
:10060000044B181C802100F03BFE031EF8D0BD46B1
:1006100003B090BD0054004080B500AF0120FFF74B
:1006200031FFBD4680BDC04680B500AF034B181CEE
:10063000012100F0C5FDBD4680BDC046005400400C
:1006400080B582B000AF78603960C020FFF79CFFB2
:100650007B68DBB2181CFFF7B9FF3B68DBB2181CE4
:10066000FFF7B4FFFFF7D8FFFFF7DEFFBD4602B08C
:1006700080BDC04690B58BB000AFF860B9607A60BD
:100680003B60786801F088FE041C386801F084FE45
:10069000031C201C191C01F077FA031C7B62786A8A
:1006A0008621C90501F0A8FB031C181C01F01EFAE5
:1006B000031C3B62BB68DA013B6AD3182F4A94469D
:1006C0006344FB617B68DA013B68396A4B43D31AA8
:1006D000BB613B687B61C020FFF756FFFB68DBB264
:1006E000181CFFF773FF7A69FF231B0213401B0AD4
:1006F000DBB2181CFFF76AFF7B69DBB2181CFFF73F
:1007000065FFFA69C0239B0213401B0CDBB2181C67
:10071000FFF75CFFFA69FF231B0213401B0ADBB2E1
:10072000181CFFF753FFFB69DBB2181CFFF74EFFE5
:100730007A69F0231B0313401B0BDAB2B969F0236B
:100740001B030B401B0CDBB21343DBB2181CFFF77F
:100750003DFFBA69FF231B0213401B0ADBB2181CC2
:10076000FFF734FFBB69DBB2181CFFF72FFFFFF761
:1007700053FFFFF759FFBD460BB090BD00FEFFFFD2
:1007800080B588B000AFF860B9607A60BB68344A61
:1007900094466344DB01FB610023BB6101237B6161
:1007A000C020FFF7F1FEFB68DBB2181CFFF70EFF5D
:1007B0007A69FF231B0213401B0ADBB2181CFFF7E8
:1007C00005FF7B69DBB2181CFFF700FFFA69C02345
:1007D0009B0213401B0CDAB27B68DBB21343DAB224
:1007E000BB68042B01D10C2300E000231343DBB2D0
:1007F000181CFFF7EBFEFA69FF231B0213401B0ACC
:10080000DBB2181CFFF7E2FEFB69DBB2181CFFF736
:10081000DDFE7A69F0231B0313401B0BDAB2B969C2
:10082000F0231B030B401B0CDBB21343DBB2181C81
:10083000FFF7CCFEBA69FF231B0213401B0ADBB291
:10084000181CFFF7C3FEBB69DBB2181CFFF7BEFE26
:10085000FFF7E2FEFFF7E8FEBD4608B080BDC046E8
:10086000FCFFFF01F0B58FB000AFF860B9602E4B10
:100870003B632E48B96801F05DF8031C7B637B6B1A
:100880000122134002D07B6B013B7B637B6BBA6818
:100890005343FB62264BBB62F86A396B01F04AF89E
:1008A000031C7B62FB6A181C396B01F0C9F80B1C36
:1008B0003B623B6ABB610023FB61BB6A3B60002378
:1008C0007B60B869F9693A687B6801F0E5F8031C58
:1008D0000C1CBB61FC613B6B1D1C00231E1CB8691A
:1008E000F9692A1C331C01F0B7F8031C0C1CBB610E
:1008F000FC61BB697B610F4BFA689200D058796A42
:100900007A69BB6AFFF7B6FE0B4BFA689200D258C1
:100910007B6B101C191C0022FFF732FF7B6A181C2E
:10092000BD460FB0F0BDC04610807D010046C32318
:10093000FFFF0F00AC290008B429000880B584B07F
:1009400000AF78607B680020191CFFF78BFF031C49
:10095000FB600D4B1B68002B04D00C4B1B68FA6826
:100960009A420DD0B1202021FFF76AFE10204F21BE
:10097000FFF766FE044B01221A60044BFA681A6006
:10098000BD4604B080BDC046140000201800002001
:1009900080B500AFB720D221FFF752FEB120202151
:1009A000FFF74EFE10204F21FFF74AFEB1208021B5
:1009B000FFF746FE11206F21FFF742FEBD4680BDC6
:1009C00080B584B000AF7860204B181C102100F077
:1009D0001BFE0F23FB1800221A7029E01B4B181C6A
:1009E000082100F011FE0F23FB181B787A689A404B
:1009F000131C8022134005D0144B181C202100F03A
:100A0000F5FD04E0114B181C202100F0FDFD0F4BFB
:100A1000181C082100F0EAFD0C4B181C082100F0FE
:100A2000F3FD0F23FB181A780F23FB1801321A70FD
:100A30000F23FB181B78072BD0D9044B181C10214F
:100A400000F0D4FDBD4604B080BDC046000400489F
:100A500090B583B000AF78600123191C7B68B84A59
:100A6000934201DC0023191CC9B27B68B54ADC0F34
:100A7000D0179A424441231CDBB20B40DBB2002B5F
:100A80000CD0B14B1B7801221343DAB2AE4B1A7073
:100A9000AD4B1B78181CFFF793FF0BE0AA4B1B789C
:100AA00001229343DAB2A84B1A70A74B1B78181C8B
:100AB000FFF786FF0123191C7B68A44A934201DCDF
:100AC0000023191CC9B27B68A14ADC0FD0179A42D7
:100AD0004441231CDBB20B40DBB2002B0CD09A4B01
:100AE0001B7802221343DAB2974B1A70964B1B788D
:100AF000181CFFF765FF0BE0934B1B780222934312
:100B0000DAB2914B1A70904B1B78181CFFF758FF04
:100B10000123191C7B688F4A934201DC0023191CB6
:100B2000C9B27B688C4ADC0FD0179A424441231C1F
:100B3000DBB20B40DBB2002B0CD0834B1B780422C2
:100B40001343DAB2804B1A707F4B1B78181CFFF7E7
:100B500037FF0BE07C4B1B7804229343DAB27A4BCD
:100B60001A70794B1B78181CFFF72AFF0123191CF8
:100B70007B687A4A934201DC0023191CC9B27B6866
:100B8000774ADC0FD0179A424441231CDBB20B405A
:100B9000DBB2002B0CD06C4B1B7808221343DAB26B
:100BA000694B1A70684B1B78181CFFF709FF0BE0A4
:100BB000654B1B7808229343DAB2634B1A70624B81
:100BC0001B78181CFFF7FCFE0123191C7B68654A83
:100BD000934201DC0023191CC9B27B68624ADC0F16
:100BE000D0179A424441231CDBB20B40DBB2002BEE
:100BF0000CD0554B1B7810221343DAB2524B1A70AB
:100C0000514B1B78181CFFF7DBFE0BE04E4B1B789B
:100C100010229343DAB24C4B1A704B4B1B78181CC2
:100C2000FFF7CEFE0123191C7B68504A934201DC7A
:100C30000023191CC9B27B684D4ADC0FD0179A42B9
:100C40004441231CDBB20B40DBB2002B0CD03E4BEB
:100C50001B7820221343DAB23B4B1A703A4B1B78B5
:100C6000181CFFF7ADFE0BE0374B1B782022934397
:100C7000DAB2354B1A70344B1B78181CFFF7A0FE04
:100C80000123191C7B683B4A934201DC0023191C99
:100C9000C9B27B68384ADC0FD0179A424441231C02
:100CA000DBB20B40DBB2002B0CD0274B1B78402271
:100CB0001343DAB2244B1A70234B1B78181CFFF72E
:100CC0007FFE0BE0204B1B7840229343DAB21E4B91
:100CD0001A701D4B1B78181CFFF772FE0123191C9C
:100CE0007B68264A934201DC0023191CC9B27B6849
:100CF000234ADC0FD0179A424441231CDBB20B403D
:100D0000DBB2002B0DD0104B1B78802252421343D4
:100D1000DAB20D4B1A700C4B1B78181CFFF750FE03
:100D20000BE0094B1B787F221340DAB2064B1A7096
:100D3000054B1B78181CFFF743FEBD4603B090BD62
:100D400000093D007F8D5B0040000020001BB700C4
:100D50009F40DD00A0636F00FF1AB700808D5B002D
:100D60009F636F00601048017FC3C901A025260062
:100D7000FF083D00A040DD005F1048013075000015
:100D80009F252600F0B58FB000AF80235B00181CB4
:100D900000F008FD031E17D09023DB05181C8021EE
:100DA00000F0F4FB031E05D0904B181C022100F04C
:100DB0002BFC04E08D4B181C022100F017FC802353
:100DC0005B00181C00F00EFD80231B01181C00F0B6
:100DD000E9FC031E17D09023DB05181C402100F00E
:100DE000D5FB031E05D0814B181C012100F0FEFB32
:100DF00004E07E4B181C012100F006FC80231B013F
:100E0000181C00F0EFFC80235B01181C00F0CAFCEA
:100E1000031E10D09023DB05181C00F0DBFB031C25
:100E2000DBB2734A1370734A0023137080235B0193
:100E3000181C00F0D7FC80231B02181C00F0B2FC29
:100E4000031E00D1CFE06B4B1B780133DBB2694A44
:100E50001370684B1B78022B00D0BFE09023DB059A
:100E6000181C012100F092FB031CDCB29023DB056F
:100E7000181C022100F08AFB031C5B00DBB2221C61
:100E80001343DCB29023DB05181C042100F07EFB29
:100E9000031C9B00DBB2221C1343DCB29023DB0556
:100EA000181C082100F072FB031CDB00DBB2221CC3
:100EB0001343DCB29023DB05181C102100F066FB05
:100EC000031C1B01DBB2221C1343DCB29023DB05A5
:100ED000181C202100F05AFB031C5B01DBB2221C12
:100EE0001343DBB2DBB2444A1370434B1B78042B31
:100EF0000AD13F4B1B781B063B63DB177B633F4BE1
:100F0000396B7A6B19605A603B4B1B78052B15D1F6
:100F1000374B1B781B04BB62DB17FB62374B5C68EB
:100F20001B68B86AF96A021C1A433A620A1C224317
:100F30007A62324B396A7A6A19605A602E4B1B7892
:100F4000062B15D12A4B1B781B02BB61DB17FB61FB
:100F50002A4B5C681B68B869F969021C1A433A613C
:100F60000A1C22437A61254B39697A6919605A60F3
:100F7000214B1B78072B29D11D4B1B78BB6000230D
:100F8000FB601E4B5C681B68B868F968021C1A435A
:100F9000151C0A1C2243161C184B1D605E60174B63
:100FA0005C681B68181C211C154A002300F074FDA6
:100FB000031C0C1C23003B6000237B60114B396831
:100FC0007A6819605A60104B01221A700A4B1B781C
:100FD0001E2B03D1064B1A780C4B1A7080231B0270
:100FE000181C00F0FFFBBD460FB0F0BD0004004828
:100FF00032000020100000203100002028000020D6
:1010000000C2EB0B38000020300000202000002040
:1010100098B500AFFFF796F9FFF7EEF9FFF754FA2E
:10102000FFF7B6FC0E4B181C022100F0EDFA0C4B3A
:10103000181C012100F0E8FA0020FFF7C1FC094B61
:101040001B781A1C084B5C681B685343181CFFF77D
:1010500075FC054B5C681B68181CFFF7F9FCEEE794
:101060000004004820000020380000200C4885467D
:10107000002103E00B4B5B58435004310A480B4BF3
:1010800042189A42F6D30A4A02E00023136004325F
:10109000084B9A42F9D300F019F9FFF7B9FFFEE7C0
:1010A00000100020842A000800000020100000200A
:1010B0001000002044000020FEE7000080B584B04E
:1010C00000AF786039600023FB607B681B680122F9
:1010D00093431A1C7B681A607B681B68FB60FB6883
:1010E000264A1340FB603B685A683B689B681B02BA
:1010F0001343FA681343FB607B68FA681A603B6825
:101100001B681F4A1A407B681A617B681B680122B2
:101110001A437B681A600023FB607B68FA689A6058
:101120007B68FA68DA603B689A693B681B6913431D
:10113000FB607B68FA689A607B689B688022120279
:101140001A437B689A603B68DB68FB607B681A68BF
:10115000FB681A437B681A607B685B68FB60FB680E
:10116000084A1340FB603B685B69FA681343FB6005
:101170007B68FA685A60BD4604B080BDFFE0CF00CE
:10118000FFFFFFF0FF7FFF0780B582B000AF786000
:101190000A1CFB1C1A70FB1C1B78002B06D07B68FA
:1011A0001B6801221A437B681A6006E07B681B6893
:1011B000012293431A1C7B681A60BD4602B080BDB1
:1011C00080B582B000AF78600A1CFB1C1A70FB1C53
:1011D0001B78002B07D07B685B688022D2011A4302
:1011E0007B685A6005E07B685B68034A1A407B684D
:1011F0005A60BD4602B080BDFFBFFFFF80B586B01C
:1012000000AFF860081C111C7B600A23FB18021C4D
:101210001A800923FB180A1C1A7000237B61FB68E3
:101220005B687B617B690E4A13407B610A23FB1874
:101230001B889B059A0D0923FB181B781904FF23B3
:101240001B040B401A437B681A433B6A13437A69B9
:1012500013437B61FB687A695A60BD4606B080BD66
:10126000009800FC80B582B000AF78600A1CFB1CBF
:101270001A70FB1C1A787B689A62BD4602B080BD6A
:1012800080B584B000AF786039600023BB600F2365
:10129000FB1800221A707B689B69BB60BB683A68C8
:1012A0001340BB60BB68002B04D00F23FB18012246
:1012B0001A7003E00F23FB1800221A700F23FB188B
:1012C0001B78181CBD4604B080BDC04680B500AF79
:1012D0001B4B1B4A126801210A431A60184B184A1B
:1012E000526818490A405A60154B154A1268164947
:1012F0000A401A60124B124A126814490A401A60D6
:101300000F4B0F4A526812490A405A600C4B0C4A64
:10131000D26A0F218A43DA62094B094A126B0D49DE
:101320000A401A63064B064A526B01218A435A63EC
:10133000034B00229A6000F00FF8BD4680BDC04606
:10134000001002400CB8FF08FFFFF6FEFFFFFBFF96
:10135000FFFFC0FFACFEFFFF80B582B000AF0023EF
:101360007B6000233B60314B304A12688021490288
:101370000A431A602D4B1A6880239B0213403B607E
:101380007B6801337B603B68002B04D17A68A02323
:10139000DB019A42EED1254B1A6880239B02134051
:1013A00002D001233B6001E000233B603B68012B3E
:1013B00038D11F4B11221A601C4B1C4A52685A60CC
:1013C0001A4B1A4A52685A60184B184A52681949FF
:1013D0000A405A60154B154A5268D02109030A4346
:1013E0005A60124B114A1268802149040A431A605C
:1013F000C0460E4B1A6880239B041340F9D00B4B58
:101400000A4A526803218A435A60084B074A5268C5
:1014100002210A435A60C046044B5B680C22134009
:10142000082BF9D1BD4602B080BDC0460010024075
:1014300000200240FFFFC0FF80B586B000AF78609B
:10144000396000237B6100233B610023FB600023A4
:101450007B617CE07B6901229A40131C3B613B6805
:101460001B683A691340FB60FA683B699A426BD18A
:101470003B681B79012B03D03B681B79022B34D1CD
:101480007B689B687A695200111C03228A40D24310
:101490001A407B689A607B689A683B685B79191C84
:1014A0007B695B0099400B1C1A437B689A607B68E0
:1014B0009B889BB27A6992B2111C01228A4092B237
:1014C000D24392B213409AB27B689A807B689B8821
:1014D0009AB23B689B79191C7B699BB299400B1CA3
:1014E0009BB213439AB27B689A807B681B687A69C7
:1014F0005200111C03228A40D2431A407B681A60B2
:101500007B681A683B681B79191C7B695B009940F2
:101510000B1C1A437B681A607B68DB687A6992B29D
:101520005200032191400A1CD2431A407B68DA60C2
:101530007B68DA683B68DB79191C7B695B00994042
:101540000B1C1A437B68DA607B6901337B617B6922
:101550000F2B00D87EE7BD4606B080BD80B582B0B7
:1015600000AF78607B68084A1A607B6800221A71B5
:101570007B6801225A717B6800229A717B68002285
:10158000DA71BD4602B080BDFFFF000080B584B0B7
:1015900000AF78600A1CBB1C1A800F23FB180022C6
:1015A0001A707B681B8A9BB2BA1C128813409BB2CC
:1015B000002B04D00F23FB1801221A7003E00F2325
:1015C000FB1800221A700F23FB181B78181CBD464D
:1015D00004B080BD80B582B000AF78607B681B8AA4
:1015E0009BB2181CBD4602B080BDC04680B582B01B
:1015F00000AF78600A1CBB1C1A80BB1C1A887B6871
:101600009A61BD4602B080BD80B582B000AF7860FF
:101610000A1CBB1C1A807B68BA1C12881A85BD463E
:1016200002B080BD80B584B000AF7860081C111C8A
:10163000BB1C021C1A807B1C0A1C1A700023FB6056
:101640000023BB607B1C1B78BA1C128807210A4050
:1016500092009340FB60BB1C1B88DB089BB2181CEC
:10166000BB1C1B88DB089BB21A1C7B6808329200EB
:10167000D358BA1C128807210A409200111C0F226D
:101680008A40D2431A40111C7B68021C0832920027
:10169000D150BB1C1B88DB089BB21A1C7B6808322C
:1016A0009200D258FB681343BB60BB1C1B88DB084D
:1016B0009BB21A1C7B6808329200B968D150BD46B3
:1016C00004B080BD80B584B000AF78600023FB60BB
:1016D000334BFB607B689B79002B4FD0304A304BFB
:1016E00019687B681B68DB430B4013602C4A2C4B4A
:1016F00059687B681B68DB430B4053607B681B7930
:101700001A1CFB689B18FB60FB68FA6811687A6812
:1017100012680A431A60224A214B99687B681B6849
:10172000DB430B4093601E4A1D4BD9687B681B68E6
:10173000DB430B40D3607B685B79102B0ED1184ADA
:10174000174B99687B681B680B439360144A144BD2
:10175000D9687B681B680B43D3601DE0104BFB60AE
:101760007B685B791A1CFB689B18FB60FB68FA6856
:1017700011687A6812680A431A600DE07B681B7969
:101780001A1CFB689B18FB60FB68FA6811687A6892
:101790001268D2430A401A60BD4604B080BDC046FC
:1017A0000004014080B584B000AF78600F23FB18BF
:1017B00000221A700A4B5B697A68134004D00F2329
:1017C000FB1801221A7003E00F23FB1800221A7085
:1017D0000F23FB181B78181CBD4604B080BDC04603
:1017E0000004014080B582B000AF7860024B7A6897
:1017F0005A61BD4602B080BD00040140B0B584B05E
:1018000000AF021CFB1D1A70BB1D0A1C1A700023BE
:10181000FB60BB1D1B78032213409B000F229A40E4
:10182000131CFB601849BB1D1B789B08DBB2181CFE
:10183000154ABB1D1B789B08DBB202339B009B58EB
:10184000FA68D2431A40831C9B005A500E48BB1DB5
:101850001B789B08DBB21D1C0B4ABB1D1B789B0829
:10186000DBB202339B009A58FB1D1978BB1D1B7815
:10187000032423409B0099400B1C1A43AB1C9B0084
:101880001A50BD4604B0B0BD0000014080B584B020
:1018900000AF78600023FB607B689B78002B39D019
:1018A000234A7B681B789B08DBB2C0339B009B58A4
:1018B000FB607B681B781A1C03231340DB00FF22AC
:1018C0009A40131CDA43FB681340FB607B685B782B
:1018D0009B01FF221A407B681B78191C03230B40D5
:1018E000DB009A40131CFA681343FB6010497B68C5
:1018F0001B789B08DBB2C0339B00FA685A500C4B34
:101900007A681278111C1F220A40012191400A1C9A
:101910001A600AE006497B681B781A1C1F231340D3
:1019200001229A40131C80228B50BD4604B080BD1A
:1019300000E100E0002243088B4274D303098B428C
:101940005FD3030A8B4244D3030B8B4228D3030C8F
:101950008B420DD3FF22090212BA030C8B4202D331
:101960001212090265D0030B8B4219D300E0090A59
:10197000C30B8B4201D3CB03C01A5241830B8B4262
:1019800001D38B03C01A5241430B8B4201D34B034B
:10199000C01A5241030B8B4201D30B03C01A5241B0
:1019A000C30A8B4201D3CB02C01A5241830A8B4235
:1019B00001D38B02C01A5241430A8B4201D34B021E
:1019C000C01A5241030A8B4201D30B02C01A524182
:1019D000CDD2C3098B4201D3CB01C01A5241830936
:1019E0008B4201D38B01C01A524143098B4201D370
:1019F0004B01C01A524103098B4201D30B01C01A9B
:101A00005241C3088B4201D3CB00C01A5241830814
:101A10008B4201D38B00C01A524143088B4201D341
:101A20004B00C01A5241411A00D2014652411046A1
:101A30007047FFE701B5002000F00CF802BDC0467A
:101A40000029F7D003B5FFF775FF0EBC4243891A92
:101A50001847C0467047C046002B11D1002A0FD14D
:101A6000002900D1002802D00021C943081C07B476
:101A7000024802A14018029003BDC046D9FFFFFFF3
:101A800003B4684601B5029800F064F8019B9E46D5
:101A900002B00CBC7047C046F0B54F464646050440
:101AA0002D0C2C1CC0B41704160C3F0C9946030CCB
:101AB0007C4375435F4373437D19260CAD199C46E7
:101AC000AF4203D980235B029846C4444B4651433E
:101AD000434324042E0C240C2D0466442C1959185D
:101AE0008919201C0CBC90469946F0BD9E2110B56A
:101AF000C905041C00F0C8FC002803D1201C00F01C
:101B00002BFC10BD9E21201CC90500F0A7FA00F097
:101B100023FC80231B069C466044F2E7F0B583B0AB
:101B2000161C1F1C0090019100F0D6FC041C0D1C1B
:101B3000221C2B1C301C391CFFF7AEFF009A019BA6
:101B4000121A8B410899201C0A604B60291C03B0B3
:101B5000F0BDC046F0B5141C83B01D1C009001916F
:101B600000F0B2FD221C2B1C061C0F1CFFF794FF7B
:101B7000009A019B121A8B410899301C0A604B6035
:101B8000391C03B0F0BDC046F0B556464D465F4621
:101B90004446F0B443024500C70F83B08A465C0A4E
:101BA0002E0EB94641D0FF2E26D080231B0423439E
:101BB000DC00002398469B467F3E53465B025D0A4D
:101BC00053465A00DB0F120E9A4639D0FF2A33D003
:101BD00080231B042B43DD0000237F3A5146B21AB9
:101BE00046467940081C01921E430F2E00D976E02C
:101BF0007E4AB6009659B746002C30D10823984645
:101C0000063B9B46D9E780230021DB03FF245B02D0
:101C1000E4055B0AC90723430B43181C03B03CBC13
:101C200090469946A246AB46F0BD002C28D104232D
:101C30009846033B9B46C0E7002D1FD1022302E0DC
:101C4000002D11D10123B21A504646467840019228
:101C50001E430F2E27D86649B60089598F460C239C
:101C60009846093B9B46A8E7281C00F017FC762203
:101C7000431F52429D40121A0023AFE70323ADE7F2
:101C8000201C00F00BFC431F9C4076235B421E1A75
:101C9000002398469B4690E70025D1469B465B462D
:101CA0004846022B6FD10121FF2401400023AEE7FB
:101CB0007E23019A5B429B1A1B2B6DDD01214B4653
:101CC000194000240023A2E78023DB031C4249D1F2
:101CD0008023DB0323435B025B0A391C96E7630125
:101CE0006D01AB4237D389461A2001215B1B0124C9
:101CF0001E1C49005B00002E01DBAB4201D35B1BC5
:101D0000214301380028F3D1581E83410B431D1C89
:101D1000019C7F34002CCBDD6B0704D00F232B40BC
:101D2000042B00D004352B0104D5019A314B8032AD
:101D3000141C1D40FE2C07DD4B460121FF241940D9
:101D4000002364E7251CAAE701214A46AB015B0A90
:101D5000E4B211405BE7019A8946013A01921B20E7
:101D60000021C4E71D4207D023435B025B0A391CF4
:101D70004CE700256302ABD58023DB032B435B02DA
:101D80005B0A514642E7032B25D0012BC0D101212C
:101D90000024014000233AE7291CD9402B1C019A5A
:101DA0009E3293405D1EAB410B435A0704D00F2275
:101DB0001A40042A00D004335A0105D54B460121AC
:101DC00001241940002322E701214A469B015B0AB6
:101DD000114000241BE7802301214A46DB032B43EB
:101DE0005B020A405B0A111C10E7C046BC290008D0
:101DF000FC290008FFFFFFF7F0B55F4656464D4649
:101E00004446F0B445024600C40F83B00F1C6D0A6F
:101E1000360EA34645D0FF2E25D080231B041D433C
:101E200000239A46ED007F3E01937B025B0A9846B1
:101E30007800FB0F000E994640D0FF2838D0802351
:101E400042461B041343DB00984600237F384A4672
:101E5000019F30186240411C1F430F2F69D87D4EEF
:101E6000BF00F659B746002D45D108230193063B24
:101E70009A46DAE793465346022B2FD15B4601245C
:101E800000251C40FF236D02DB056D0AE4071D439E
:101E90002543281C03B03CBC90469946A246AB465D
:101EA000F0BD002D2CD104230193033B9A46BCE7DF
:101EB00043465A4253410322D31AC8E742460123FC
:101EC000002AC4D0404600F0E9FA4246431F9A4037
:101ED00076235B42181A90460023B8E7032B00D103
:101EE000ADE0012B00D08CE05B4654461C40E4B2D0
:101EF00000230025C7E70C230193093B9A4694E78A
:101F0000281C00F0CBFA7626431F9D400023764222
:101F1000361A01939A4688E780250024ED03FF23B3
:101F2000B1E74546CB469A46A5E7454693469A46CD
:101F3000A1E743462C041B0C9C46230C4446260474
:101F40001C1C360C2F0C7443351C66467D437343B2
:101F50007743EB18260C9E19B54203D980235B0208
:101F60009C46674424043304240C1B199D016C1EF9
:101F7000A5419B0E360C2B43BD19AD011D432B0112
:101F800004D5012368081D400543081C031C7F334A
:101F9000002B2CDD690704D00F212940042900D033
:101FA0000435290103D52C4B1D40031C8033FE2B27
:101FB00017DD0124FF231440002564E78020C003BF
:101FC000054209D04346034206D1454605436D020A
:101FD0006D0A4C46FF2356E705436D026D0AFF2349
:101FE00051E70124AD016D0ADBB214404BE77E23BB
:101FF0005B421B1A1B2B07DD012400231440002524
:1020000041E7081C5A46C1E79E30291C8540D9404B
:10201000681E85410D436B0704D00F232B40042B12
:1020200000D004356B0104D50124012314400025A0
:1020300029E70124AD016D0A1440002323E7802322
:10204000DB031D4301245B466D0223401C1C6D0A0B
:10205000FF2318E73C2A0008FFFFFFF7F8B54A0006
:10206000430244004D02C00F240E061C9B09120EB1
:10207000C90FAD09FF2A00D175E0012779408842D8
:1020800050D0A01A002800DC8FE0002A1ED1002DBD
:1020900000D075E05A0704D00F221A40042A00D05D
:1020A000043380220120D2041A403040002A32D06A
:1020B0000134FF2C00D184E09B015B0AE4B25B0297
:1020C000E4055B0A2343C0071843F8BDFF2CE1D0A9
:1020D0008022D20415431B287ADD01255B1B5A019F
:1020E0005DD59B019F09381C00F0D8F90538874061
:1020F000844269DC001B1F243A1C431C201ADA406E
:102100008740131C7C1EA74100243B43C2E7131EDB
:1021100045D100230020DB08FF2C28D05B025B0A9E
:10212000E4B2CCE7A11A00295BDD002A2ED0FF2CF7
:10213000B0D08022D20415431B2974DC2F1C20222E
:10214000CF40511A8D40691E8D413D435B195A01A4
:1021500025D50134FF2C74D001217E4A194013404B
:102160005B080B4396E7002D00D088E785E7002B3E
:1021700027D08022D20313435B025B0AFF249EE731
:1021800001380028AAD0FF2CA5D183E7002D00D16B
:1021900080E701390029D9D0FF2CCDD17AE75A0741
:1021A00000D079E701203040B5E7002825D1621C36
:1021B000D2B2012A55DD5F1B7A012DD5EF1A0E1C14
:1021C00091E7FF2400237AE7624B241A3B4061E742
:1021D000291C2022C140101A8540681E85410D43EC
:1021E0007CE7002946D1621CD1B201292BDDFF2AF0
:1021F00026D0EB185B08141C4CE7002C15D0FF2AE6
:102200001AD08024E404404223431B284DDD0123DF
:10221000EB1A141C0E1C62E7002F00D063E70023AA
:102220000020002477E7012590E7002B39D0C04338
:102230000028EDD0FF2AE8D12B1CFF240E1C29E733
:10224000FF24002367E7002C5AD1002B7FD0002DFC
:1022500000D11FE75B195A01A1D53E4A0134134052
:1022600018E7002C15D1002B2FD1002D5ED02B1C90
:102270000E1C0FE7002C21D1002B54D0C94300299C
:1022800004D0FF2A4CD01B2958DD01235B19141CF4
:102290005DE7002B23D1002D4BD02B1C0E1CFF24FF
:1022A000F8E62B1C141C0E1CF4E61E1C2024C64051
:1022B000201A8340581E83413343A9E7FF2A2FD0B9
:1022C0008024E40449422343DDE7002D00D1E1E608
:1022D0005A1B500100D41AE7EB1A0E1CDAE6FF2451
:1022E000002D00D1D6E68022DB08D203134204D0B1
:1022F000ED08154201D12B1C0E1CDB00FF24C9E6A2
:10230000002B0DD0FF24002D00D1C3E68022DB0876
:10231000D2031342F1D0ED081542EED12B1CECE7AD
:102320002B1CFF24B6E62B1C141CB3E6231C002038
:10233000F1E6802300209B04FF24ECE61F1C2024F0
:10234000CF40611A8B40591E8B413B439EE72B1CAB
:10235000A0E6C046FFFFFFFB4202510A4200C30F46
:10236000120E00207E2A0DDD9D2A0CDC8020000448
:102370000143952A0ADC9620821AD1400A1C584251
:102380004240D0187047034A9818FBE7963A9140AC
:102390000A1CF4E7FFFFFF7F10B5041E35D000F0E4
:1023A0007DF89E21091A962909DC082830DD021CD7
:1023B000231C083A93405B025B0AC8B220E09929CB
:1023C0000CDD0522231C121AD3401A1C031C1B33DC
:1023D0009C40231C5C1EA34113431C1C052801DDEB
:1023E000431F9C400F4B2340620704D00F22144030
:1023F000042C00D004335A010ED49B015B0AC8B2EE
:102400005B025B0AC005184310BD00200023F7E7FC
:1024100063025B0AC8B2F3E79F21024A091A13401C
:10242000EBE7C046FFFFFFFB8446081C6146FFE761
:102430001FB500F069FA002801D40021C8421FBD71
:1024400010B500F0EDF94042013010BD10B500F0BC
:102450005BFA002801DB002010BD012010BDC04642
:1024600010B500F051FA002801DD002010BD012058
:1024700010BDC04610B500F0FDF9002801DC0020B9
:1024800010BD012010BDC04610B500F0F3F90028C2
:1024900001DA002010BD012010BDC0461C2101231F
:1024A0001B04984201D3000C10391B0A984201D337
:1024B000000A08391B09984201D30009043902A215
:1024C000105C40187047C04604030202010101017C
:1024D0000000000000000000F0B544465F4656468C
:1024E0004D46F0B41C1C85B0002900DAA9E00F1C91
:1024F0000021061C8846101C191C002C00DA97E0ED
:10250000341C3D1C82468946B94273D870D0494676
:10251000504600F03FFA8346391C301C00F03AFA6E
:102520005B46181A031C8346203B9C4600D59CE062
:102530000023002251460092019363469940019185
:1025400051468140019B0091BB4200D983E000D1FC
:102550007EE0009A019B341C3D1CA41A9D416346F9
:10256000002B00DA9AE00026002702960397013636
:102570009E400396012686400296002800D171E015
:102580000099019AD30799464B464E081E435708B7
:10259000002301220CE0AF4201D1A6420AD8A41BBD
:1025A000BD4124196D410138A4185D41002806D0B1
:1025B000AF42F0D9013824196D410028F8D120220A
:1025C000029E039F5B46524236196F4199185AD4B6
:1025D000281CC8402C1C5B46DC40002968DB041C1E
:1025E0008C40231C59468840021CB61A9F4103E0C8
:1025F000B0428CD90026002741464B1E994100234A
:1026000000910193009A019B002554429D41331C87
:102610006340181C3B1C6B40191C009B019CC0189C
:10262000614105B03CBC90469946A246AB46F0BD20
:102630004346DB430C1C9846131C00215842A14121
:102640005EE7002746428F4101214942884652E712
:10265000B14200D87DE700260027029603970028A4
:1026600000D08DE7029E039FC6E720215346091A3A
:10267000CB400022191C0023009201934B4683405B
:102680000B4301935CE75A4620239B1A2A1C9A406D
:10269000201C131C5A46D04018439BE720260027D5
:1026A000331A0026029603970127DF40039761E75C
:1026B0005B4620215D46C91A031CAC40CB40191C67
:1026C000231C0B438EE7C046F0B545464E465746A1
:1026D000E0B4041C82B00D1C914698468B4262D82F
:1026E0005FD04146484600F055F9291C061C201CC5
:1026F00000F050F92023311A5B428A46C81865D48D
:102700004B4683401F1C4B468B401E1CAF4258D883
:1027100055D0A41BBD41002800DA77E00022002339
:102720000092019301328240019201238B40009379
:1027300000293CD0FB079846404672087B080243BC
:10274000012600270CE0AB4201D1A2420AD8A41A0C
:102750009D4124196D410139A4197D41002906D0FC
:10276000AB42F0D9013924196D410029F8D120225A
:102770000098019953465242001969419E183AD473
:102780002F1CF7405346DD40002E29DB3C1CB44093
:10279000231C5446A7403A1C801A9941009001918D
:1027A00005E082429DD90023002400930194009803
:1027B000019902B01CBC90469946A246F0BDA342C6
:1027C000A7D90022002300920193B1E720224B46B3
:1027D000521AD3401A1C43468B401F1C174392E7E2
:1027E000534620245646E41A3B1CB540E3401C1CCB
:1027F0002B1C2343CDE7524620239B1A2A1C9A40C8
:10280000271C131C5246D7401F43BBE7202300223E
:10281000581A0023009201930132C240019284E7CA
:10282000430270B542004C005D0AC30F4802120E0D
:10283000460A240EC90FFF2A05D0FF2C08D001201C
:10284000A2420BD070BD0120002DFBD1FF2CF6D190
:102850000120002EF6D10120A242F3D1B542F1D1E0
:102860008B4205D0002AEDD1281C431E9841E9E790
:102870000020E7E7F0B543024D024A0044005E0A3B
:10288000240EC30F6D0A120EC90FFF2C0DD0FF2AA4
:1028900031D0002C0DD177427741002A23D1002D71
:1028A00021D10020002F0BD107E0002E28D1FF2AD4
:1028B00021D0002A05D08B4207D05842012318436B
:1028C000F0BD002DF9D08B42F7D19442F5DC04DB4A
:1028D000AE42F2D80020AE42F2D25842434101202B
:1028E0005B421843ECE7002FE5D04842414101200C
:1028F00049420843E4E7002D02D1002CCBD0DAE7AF
:1029000002204042DCE7C0464302F0B542004C00E2
:102910005E0AC30F4802120E450A240EC90FFF2A91
:102920000FD0FF2C1AD0002A10D177427741002C0B
:1029300029D0002F17D04842414101204942084385
:102940000BE00220002E08D1FF2C07D0002C0AD16A
:10295000002D08D1584201231843F0BD0220002D5C
:10296000FBD1002AE1D08B42F4D1A242F2DC04DB9D
:10297000AE42EFD80020AE42EFD258424341012090
:102980005B421843E9E7002DD3D10020002FE4D1AA
:10299000E0E7C04610B5002903D1FFF77FFD2030E6
:1029A00002E0081CFFF77AFD10BDC0461A000000C7
:1029B000220000002A00000032000000DE1C000897
:1029C000A61C0008C21C00089A1C0008C21C0008B3
:1029D000061C0008C21C00089A1C0008A61C00085F
:1029E000A61C0008061C00089A1C0008441D0008CC
:1029F000441D0008441D0008C81C0008A61C00084F
:102A0000A61C00088E1D0008981C00088E1D0008DA
:102A1000061C00088E1D0008981C0008A61C000853
:102A2000A61C0008061C0008981C0008441D00088D
:102A3000441D0008441D0008721D0008321F0008D4
:102A40002A1F00082A1F0008221F0008741E000801
:102A5000741E0008181F0008221F0008741E0008BA
:102A6000181F0008741E0008221F0008761E0008A8
:0C2A7000761E0008761E0008BC1F00083F
:082A7C005CFAFF7F010000007D
:102A84000000000001020304010203040607080910
:0400000508000000EF
:00000001FF
